:020000040000FA
:02000000F72ADD
:08000800F100030EF000831665
:1000100003138C1E0F28831203138C1A18288316BF
:1000200003130C1E1728831203130C1A6E287F2843
:1000300083120313F60A1A08F20001307602031D38
:1000400039287208F300AA307302031967280130B7
:100050007302031967280230730203196728A1305D
:10006000730203196728A230730203196728F60187
:10007000672802307602031D40287208F4006728C2
:100080007208F500F601AA307302031D4928842086
:10009000602801307302031D51280521F701F80182
:1000A000602802307302031D59287D21F701F801F1
:1000B0006028A1307302031D5F28F5216028762295
:1000C000F901831603130C16831203136728831296
:1000D0000313981C0F28181218160F28F90A01305C
:1000E0007902031D76287708990017287808990067
:1000F000831603130C1283120313F9011728700ED1
:100100008300F10E710E0900861706130000061019
:100110000617000006130000061406170000061359
:10012000000006100617000006130000061406174C
:10013000000006130000061006170000061300005A
:10014000061406170000061300000610061700002C
:1001500006130000061406170000831603133F3031
:100160008600831203130613000006187814061C79
:10017000781006170000061300000618F814061C75
:10018000F810061700000613000006187815061C64
:10019000781106170000061300000618F815061C53
:1001A000F811061700000613000006187816061C42
:1001B000781206170000061300000618F816061C31
:1001C000F812061700000613000006187817061C20
:1001D000781306170000061300000618F817061C0F
:1001E000F8130617000006130000F701061877142D
:1001F000061C7710061700008613000083160313F1
:100200003E30860083120313080006178617061374
:10021000000006140617000006130000061006175B
:100220000000061300000610061700000613000069
:10023000061006170000061300000610061700003F
:100240000613000006100617000006130000061033
:10025000061700000613000006100617000006131C
:10026000000075180614751C06100617000006130A
:100270000000F5180614F51C0610061700000613FA
:10028000000075190614751D0610061700000613E8
:100290000000F5190614F51D0610061700000613D8
:1002A0000000751A0614751E0610061700000613C6
:1002B0000000F51A0614F51E0610061700000613B6
:1002C0000000751B0614751F0610061700000613A4
:1002D0000000F51B0614F51F061006170000061394
:1002E000000074180614741C06100617000086130C
:1002F00081010B110B1D7A290800061786170613BA
:10030000000006100617000006130000061406176A
:100310000000061300000610061700000613000078
:10032000061006170000061300000610061700004E
:100330000613000006100617000006130000061042
:10034000061700000613000006100617000006132B
:10035000000075180614751C061006170000061319
:100360000000F5180614F51C061006170000061309
:10037000000075190614751D0610061700000613F7
:100380000000F5190614F51D0610061700000613E7
:100390000000751A0614751E0610061700000613D5
:1003A0000000F51A0614F51E0610061700000613C5
:1003B0000000751B0614751F0610061700000613B3
:1003C0000000F51B0614F51F0610061700000613A3
:1003D000000074180614741C06100617000086131B
:1003E00081010B110B1DF22908008617061300006E
:1003F000061406170000061300000610061700007A
:100400000613000006100617000006130000061071
:10041000061700000613000006100617000006135A
:100420000000061406170000061300000610061749
:1004300000000613000006140617000083160313BD
:100440003F30860083120313061300000618781449
:10045000061C781006170000061300000618F81492
:10046000061CF81006170000061300000618781581
:10047000061C781106170000061300000618F81570
:10048000061CF8110617000006130000061878165F
:10049000061C781206170000061300000618F8164E
:1004A000061CF8120617000006130000061878173D
:1004B000061C781306170000061300000618F8172C
:1004C000061CF8130617000006130000F7010618B3
:1004D0007714061C77100617000086130000831699
:1004E00003133E3086008312031308008617061399
:1004F0000000061006170000061300000614061779
:100500000000061300000610061700000613000086
:10051000061006170000061300000610061700005C
:10052000061300000614061700000613000006104C
:1005300006170000061300000614061700008316B5
:1005400003133F30860083120313061300000618BE
:100550007814061C78100617000006130000061811
:10056000F814061CF8100617000006130000061801
:100570007815061C781106170000061300000618EF
:10058000F815061CF81106170000061300000618DF
:100590007816061C781206170000061300000618CD
:1005A000F816061CF81206170000061300000618BD
:1005B0007817061C781306170000061300000618AB
:1005C000F817061CF8130617000006130000F701C1
:1005D00006187714061C7710061700008613000013
:1005E000831603133E308600831203130800831220
:1005F00003138501860107309F0083160313D7304C
:100600008100FF3085003E30860081309900243023
:100610009800831203139030980085018601F6013B
:10062000F901831603138B170B178C160C12831208
:10063000031306178617061300000610061700009E
:10064000061300000610061700000613000006142B
:100650000617000006130000061406170000061314
:10066000000006100617000006130000061006170B
:100670000000061300000610061700000613000015
:1006800006100617000006130000061006170000EB
:1006900006130000061406170000061300000610DB
:1006A00006170000061300000610061700000613C8
:1006B00000000610061700000613000006100617BB
:1006C00000000613000006100617000006130000C5
:1006D000061006170000861381010B110B1D6E2BEF
:1006E0008617061300000610061700000613000008
:1006F0000614061700000613000006140617000073
:10070000061300000614061700000613000006106A
:100710000617000006130000061406170000061353
:100720000000061406170000061300000614061742
:0A0730000000861300009C2B9C2B98
:02400E00623F0F
:00000001FF
